:1000000012C01895A8CC189518951895189518959C
:100010001895189518951895189518951895189578
:100020001895189518958FE58DBFC0E4E6E24E2E21
:1000300084E08EBFD4E0F4E05F2EA89584B7082E4C
:10004000877F84BF88E1992781BD91BDEEEFF3E002
:10005000A0E6B0E088278D933197E9F783E389B96B
:1000600080E080BD88E18AB9662480E087BB7FEFAD
:1000700078BB8FEF84BB7FEF75BB8E98969A8D9877
:10008000959A8998919A78947BB770687BBF86DB44
:1000900080EA90E0A0E6B0E08D939C938EE190E042
:1000A000A2E6B0E08D939C9377EF75BBA0E3B0E040
:1000B0000C9101FB81E00EF080E08F93A0E3B0E0B3
:1000C0000C9105FB81E00EF480E09F9189238F93D2
:1000D000A0E3B0E00C9106FB81E00EF080E09F9180
:1000E0008923882309F40FC0EEEFF6E144DC06B360
:1000F0000E3F09F003C0E4ECF5E13DDC859B03C055
:10010000EAEFF6E138DC7FED75BBA0E3B0E00C91DF
:1001100001FB81E00EF080E08F93A0E3B0E00C9152
:1001200005FB81E00EF080E09F9189238F93A0E38F
:10013000B0E00C9106FB81E00EF080E09F918923F6
:10014000882309F480C006B30E3F09F008C0E4E636
:10015000F7E111DCA0E6B0E08D919C9110DB06B3D5
:100160000D3F09F008C0E0E6F7E105DCA0E6B0E0ED
:100170008D919C9104DB06B30B3F09F008C0ECE5C0
:10018000F7E1F9DBA0E6B0E08D919C91F8DA06B3D7
:10019000073F09F008C0E8E5F7E1EDDBA0E6B0E0D5
:1001A0008D919C91ECDA06B30F3E09F00DC0E0E5AD
:1001B000F7E1E1DBA0E6B0E08D919C91E0DAA0E60A
:1001C000B0E08D919C91DBDA06B30F3D09F011C0D0
:1001D000E0E3F7E1D0DBBBD906B30F3D09F4F8CF7C
:1001E000E0E4F7E1C8DB80E090E0A4E6B0E08D93C6
:1001F0009C9306B30F3B09F011C0ECE2F7E1BBDBC7
:10020000A6D906B30F3B09F4F8CFECE3F7E1B3DB73
:1002100080E090E0A4E6B0E08D939C9306B30F37A6
:1002200009F011C0E8E2F7E1A6DB91D906B30F3778
:1002300009F4F8CFE8E3F7E19EDB80E090E0A4E684
:10024000B0E08D939C9386990CC006B30F3E09F0E5
:1002500003C0E8E6F7E18FDBA0E6B0E08D919C916A
:100260008EDAA0E3B0E00C9101FB81E00EF080E0BB
:100270008F93A0E3B0E00C9105FB81E00EF480E0E9
:100280009F9189238F93A0E3B0E00C9106FB81E05E
:100290000EF080E09F918923882309F424C0EEEFBB
:1002A000F6E169DB06B30E3F09F003C0E0E2F7E1D7
:1002B00062DB06B30D3F09F003C0E8E1F7E15BDB69
:1002C00006B30B3F09F003C0E0E1F7E154DB06B3EE
:1002D000073F09F003C0E8E0F7E14DDB859B03C071
:1002E000EAEFF6E148DB7EEF75BB869951C006B3B5
:1002F0000D3F09F017C0E4EFF6E13DDBE0ECF5E17E
:100300003ADB25D906B30D3F09F4F8CFE4EFF5E168
:1003100032DBE6EFF6E12FDB80E090E0A4E6B0E030
:100320008D939C9306B30B3F09F017C0E4EFF6E101
:1003300022DBE0EEF5E11FDB0AD906B30B3F09F43F
:10034000F8CFE4E3F6E117DBE6EFF6E114DB80E05B
:1003500090E0A4E6B0E08D939C9306B30F3D09F0C6
:1003600017C0E4EFF6E107DBEEEDF5E104DBEFD8D3
:1003700006B30F3D09F4F8CFE0E3F6E1FCDAE6EF6F
:10038000F6E1F9DA80E090E0A4E6B0E08D939C938A
:10039000A0E3B0E00C9101FB81E00EF080E08F93D0
:1003A000A0E3B0E00C9105FB81E00EF080E09F91AE
:1003B00089238F93A0E3B0E00C9106FB81E00EF05F
:1003C00080E09F918923882309F49CC006B30E3FE7
:1003D00009F00EC0E4E5F7E1CEDAB9D806B30E3F76
:1003E00009F4F8CF80E090E0A4E6B0E08D939C9310
:1003F00006B30D3F09F011C0E0ECF5E1BCDAA7D877
:1004000006B30D3F09F4F8CFE4EFF5E1B4DA80E08C
:1004100090E0A4E6B0E08D939C9306B30B3F09F007
:1004200011C0E0EEF5E1A7DA92D806B30B3F09F46C
:10043000F8CFE4E3F6E19FDA80E090E0A4E6B0E0F4
:100440008D939C9306B3073F09F011C0E6E8F5E1F0
:1004500092DA7DD806B3073F09F4F8CFECE9F5E16D
:100460008ADA80E090E0A4E6B0E08D939C9306B336
:100470000F3E09F011C0E4E8F5E17DDA68D806B373
:100480000F3E09F4F8CFE8E9F5E175DA80E090E095
:10049000A4E6B0E08D939C9306B30F3D09F011C024
:1004A000EEEDF5E168DA53D806B30F3D09F4F8CF65
:1004B000E0E3F6E160DA80E090E0A4E6B0E08D935E
:1004C0009C9306B30F3B09F011C0E4E3F7E153DA64
:1004D0003ED806B30F3B09F4F8CFE4E4F7E14BDA7A
:1004E00080E090E0A4E6B0E08D939C9306B30F37D4
:1004F00009F008C0ECE4F7E13EDAA0E6B0E08D9147
:100500009C913DD9819948C006B30B3F09F00EC0BC
:10051000EAEAF6E130DA1BD806B30B3F09F4F8CF6C
:1005200080E090E0A4E6B0E08D939C9306B3073F93
:1005300009F017C0EEEEF6E11EDAE6E8F5E11BDAA7
:1005400006D806B3073F09F4F8CFECE9F5E113DA72
:10055000E0EFF6E110DA80E090E0A4E6B0E08D9301
:100560009C9306B30F3E09F017C0EEEEF6E103DAF6
:10057000E4E8F5E100DAEBD706B30F3E09F4F8CF73
:10058000E8E9F5E1F8D9E0EFF6E1F5D980E090E0AF
:10059000A4E6B0E08D939C937DEF75BB869987C0F0
:1005A00006B30E3F09F017C0E4EFF6E1E4D9E0EF3F
:1005B000F5E1E1D9CCD706B30E3F09F4F8CFE4E575
:1005C000F6E1D9D9E6EFF6E1D6D980E090E0A4E6ED
:1005D000B0E08D939C9306B30D3F09F017C0E4EF94
:1005E000F6E1C9D9E4EEF5E1C6D9B1D706B30D3FBE
:1005F00009F4F8CFECE3F6E1BED9E6EFF6E1BBD9BA
:1006000080E090E0A4E6B0E08D939C9306B30B3FAE
:1006100009F017C0E4EFF6E1AED9ECEEF5E1ABD9A5
:1006200096D706B30B3F09F4F8CFECE4F6E1A3D973
:10063000E6EFF6E1A0D980E090E0A4E6B0E08D938B
:100640009C9306B30F3D09F017C0E4EFF6E193D990
:10065000ECEDF5E190D97BD706B30F3D09F4F8CF67
:10066000ECE2F6E188D9E6EFF6E185D980E090E0AA
:10067000A4E6B0E08D939C9306B30F3B09F017C03E
:10068000E4EFF6E178D9E6EDF5E175D960D706B388
:100690000F3B09F4F8CFE0E2F6E16DD9E6EFF6E1C1
:1006A0006AD980E090E0A4E6B0E08D939C93A0E34B
:1006B000B0E00C9101FB81E00EF080E08F93A0E3AD
:1006C000B0E00C9105FB81E00EF080E09F91892362
:1006D0008F93A0E3B0E00C9106FB81E00EF080E088
:1006E0009F918923882309F4A5C006B30E3F09F022
:1006F00011C0E0EFF5E13FD92AD706B30E3F09F468
:10070000F8CFE4E5F6E137D980E090E0A4E6B0E088
:100710008D939C9306B30D3F09F011C0E4EEF5E113
:100720002AD915D706B30D3F09F4F8CFECE3F6E16B
:1007300022D980E090E0A4E6B0E08D939C9306B3CC
:100740000B3F09F011C0ECEEF5E115D900D706B367
:100750000B3F09F4F8CFECE4F6E10DD980E090E02E
:10076000A4E6B0E08D939C9306B3073F09F011C057
:10077000E8E8F5E100D9EBD606B3073F09F4F8CF76
:10078000E0EAF5E1F8D880E090E0A4E6B0E08D93EF
:100790009C9306B30F3E09F011C0E6E9F5E1EBD8F2
:1007A000D6D606B30F3E09F4F8CFECEBF5E1E3D86B
:1007B00080E090E0A4E6B0E08D939C9306B30F3DFB
:1007C00009F011C0ECEDF5E1D6D8C1D606B30F3D66
:1007D00009F4F8CFECE2F6E1CED880E090E0A4E6B0
:1007E000B0E08D939C9306B30F3B09F011C0E6ED8A
:1007F000F5E1C1D8ACD606B30F3B09F4F8CFE0E27F
:10080000F6E1B9D880E090E0A4E6B0E08D939C9347
:1008100006B30F3709F00EC0E8E4F7E1ACD897D67D
:1008200006B30F3709F4F8CF80E090E0A4E6B0E01B
:100830008D939C9381997EC006B30E3F09F00EC044
:10084000ECEDF6E198D883D606B30E3F09F4F8CF65
:1008500080E090E0A4E6B0E08D939C9306B30D3F5A
:1008600009F00EC0E6EBF6E186D871D606B30D3F6F
:1008700009F4F8CF80E090E0A4E6B0E08D939C937B
:1008800006B30B3F09F00EC0ECECF6E174D85FD66E
:1008900006B30B3F09F4F8CF80E090E0A4E6B0E0A7
:1008A0008D939C9306B3073F09F017C0EEEEF6E177
:1008B00062D8E8E8F5E15FD84AD606B3073F09F405
:1008C000F8CFE0EAF5E157D8E0EFF6E154D880E060
:1008D00090E0A4E6B0E08D939C9306B30F3E09F040
:1008E00017C0EEEEF6E147D8E6E9F5E144D82FD699
:1008F00006B30F3E09F4F8CFECEBF5E13CD8E0EF9E
:10090000F6E139D880E090E0A4E6B0E08D939C93C6
:1009100006B30F3D09F00EC0E2EAF6E12CD817D677
:1009200006B30F3D09F4F8CF80E090E0A4E6B0E014
:100930008D939C937BEF75BB8699A2C006B30E3F47
:1009400009F017C0E4EFF6E116D8EEEEF5E113D8A2
:10095000FED506B30E3F09F4F8CFE0E5F6E10BD87B
:10096000E6EFF6E108D880E090E0A4E6B0E08D93F1
:100970009C9306B30D3F09F017C0E4EFF6E1FBD7F7
:10098000E6ECF5E1F8D7E3D506B30D3F09F4F8CF6F
:10099000E0E0F6E1F0D7E6EFF6E1EDD780E090E0B9
:1009A000A4E6B0E08D939C9306B30B3F09F017C00B
:1009B000E4EFF6E1E0D7E8ECF5E1DDD7C8D506B322
:1009C0000B3F09F4F8CFE4E0F6E1D5D7E6EFF6E126
:1009D000D2D780E090E0A4E6B0E08D939C9306B37C
:1009E0000F3D09F017C0E4EFF6E1C5D7E0EDF5E102
:1009F000C2D7ADD506B30F3D09F4F8CFE4E1F6E177
:100A0000BAD7E6EFF6E1B7D780E090E0A4E6B0E031
:100A10008D939C9306B30F3B09F017C0E4EFF6E10A
:100A2000AAD7E4EDF5E1A7D792D506B30F3B09F4B9
:100A3000F8CFECE1F6E19FD7E6EFF6E19CD780E056
:100A400090E0A4E6B0E08D939C9306B30F3709F0D5
:100A500017C0E4EFF6E18FD7E8EDF5E18CD777D555
:100A600006B30F3709F4F8CFE4E2F6E184D7E6EFF6
:100A7000F6E181D780E090E0A4E6B0E08D939C930E
:100A8000A0E3B0E00C9101FB81E00EF080E08F93D9
:100A9000A0E3B0E00C9105FB81E00EF080E09F91B7
:100AA00089238F93A0E3B0E00C9106FB81E00EF068
:100AB00080E09F918923882309F4A8C006B30E3FE4
:100AC00009F011C0EEEEF5E156D741D506B30E3F61
:100AD00009F4F8CFE0E5F6E14ED780E090E0A4E637
:100AE000B0E08D939C9306B30D3F09F011C0E6EC86
:100AF000F5E141D72CD506B30D3F09F4F8CFE0E07E
:100B0000F6E139D780E090E0A4E6B0E08D939C93C5
:100B100006B30B3F09F011C0E8ECF5E12CD717D56F
:100B200006B30B3F09F4F8CFE4E0F6E124D780E008
:100B300090E0A4E6B0E08D939C9306B3073F09F0E4
:100B400011C0EAE8F5E117D702D506B3073F09F46B
:100B5000F8CFE4EAF5E10FD780E090E0A4E6B0E05A
:100B60008D939C9306B30F3E09F011C0E4E9F5E1C3
:100B700002D7EDD406B30F3E09F4F8CFE8EBF5E168
:100B8000FAD680E090E0A4E6B0E08D939C9306B3A3
:100B90000F3D09F011C0E0EDF5E1EDD6D8D406B374
:100BA0000F3D09F4F8CFE4E1F6E1E5D680E090E00E
:100BB000A4E6B0E08D939C9306B30F3B09F011C0FF
:100BC000E4EDF5E1D8D6C3D406B30F3B09F4F8CF72
:100BD000ECE1F6E1D0D680E090E0A4E6B0E08D93C1
:100BE0009C9306B30F3709F011C0E8EDF5E1C3D6C9
:100BF000AED406B30F3709F4F8CFE4E2F6E1BBD682
:100C000080E090E0A4E6B0E08D939C938199A2C02F
:100C100006B30E3F09F00EC0E4EDF6E1ACD697D472
:100C200006B30E3F09F4F8CF80E090E0A4E6B0E010
:100C30008D939C9306B30D3F09F00EC0E4E6F6E1F8
:100C40009AD685D406B30D3F09F4F8CF80E090E042
:100C5000A4E6B0E08D939C9306B30B3F09F00EC061
:100C6000EAE6F6E188D673D406B30B3F09F4F8CF71
:100C700080E090E0A4E6B0E08D939C9306B3073F3C
:100C800009F017C0EEEEF6E176D6EAE8F5E173D6A4
:100C90005ED406B3073F09F4F8CFE4EAF5E16BD67A
:100CA000E0EFF6E168D680E090E0A4E6B0E08D9356
:100CB0009C9306B30F3E09F017C0EEEEF6E15BD64B
:100CC000E4E9F5E158D643D406B30F3E09F4F8CF72
:100CD000E8EBF5E150D6E0EFF6E14DD680E090E0AC
:100CE000A4E6B0E08D939C9306B30F3D09F00EC0CF
:100CF000E8E7F6E140D62BD406B30F3D09F4F8CF70
:100D000080E090E0A4E6B0E08D939C9306B30F3BA7
:100D100009F00EC0E6E8F6E12ED619D406B30F3B73
:100D200009F4F8CF80E090E0A4E6B0E08D939C93C6
:100D300006B30F3709F00EC0E0E9F6E11CD607D480
:100D400006B30F3709F4F8CF80E090E0A4E6B0E0F6
:100D50008D939C9377EF75BB8699A2C006B30E3F27
:100D600009F017C0E4EFF6E106D6E4ECF5E103D6AE
:100D7000EED306B30E3F09F4F8CFECEFF5E1FBD567
:100D8000E6EFF6E1F8D580E090E0A4E6B0E08D93E0
:100D90009C9306B30D3F09F017C0E4EFF6E1EBD5E5
:100DA000EAECF5E1E8D5D3D306B30D3F09F4F8CF6B
:100DB000E8E0F6E1E0D5E6EFF6E1DDD580E090E0B1
:100DC000A4E6B0E08D939C9306B30B3F09F017C0E7
:100DD000E4EFF6E1D0D5E2EEF5E1CDD5B8D306B338
:100DE0000B3F09F4F8CFE8E3F6E1C5D5E6EFF6E10D
:100DF000C2D580E090E0A4E6B0E08D939C9306B36A
:100E00000F3D09F017C0E4EFF6E1B5D5E8EEF5E1E6
:100E1000B2D59DD306B30F3D09F4F8CFE4E4F6E173
:100E2000AAD5E6EFF6E1A7D580E090E0A4E6B0E031
:100E30008D939C9306B30F3B09F017C0E4EFF6E1E6
:100E40009AD5E2EDF5E197D582D306B30F3B09F4CD
:100E5000F8CFE8E1F6E18FD5E6EFF6E18CD580E05A
:100E600090E0A4E6B0E08D939C9306B30F3709F0B1
:100E700017C0E4EFF6E17FD5EAEDF5E17CD567D365
:100E800006B30F3709F4F8CFE8E2F6E174D5E6EFE0
:100E9000F6E171D580E090E0A4E6B0E08D939C93FC
:100EA000A0E3B0E00C9101FB81E00EF080E08F93B5
:100EB000A0E3B0E00C9105FB81E00EF080E09F9193
:100EC00089238F93A0E3B0E00C9106FB81E00EF044
:100ED00080E09F918923882309F4A8C006B30E3FC0
:100EE00009F011C0E4ECF5E146D531D306B30E3F6D
:100EF00009F4F8CFECEFF5E13ED580E090E0A4E610
:100F0000B0E08D939C9306B30D3F09F011C0EAEC5D
:100F1000F5E131D51CD306B30D3F09F4F8CFE8E075
:100F2000F6E129D580E090E0A4E6B0E08D939C93B3
:100F300006B30B3F09F011C0E2EEF5E11CD507D373
:100F400006B30B3F09F4F8CFE8E3F6E114D580E0EF
:100F500090E0A4E6B0E08D939C9306B3073F09F0C0
:100F600011C0ECE8F5E107D5F2D206B3073F09F46A
:100F7000F8CFE8EAF5E1FFD480E090E0A4E6B0E045
:100F80008D939C9306B30F3E09F011C0E2E9F5E1A1
:100F9000F2D4DDD206B30F3E09F4F8CFE4EBF5E16D
:100FA000EAD480E090E0A4E6B0E08D939C9306B391
:100FB0000F3D09F011C0E8EEF5E1DDD4C8D206B36B
:100FC0000F3D09F4F8CFE4E4F6E1D5D480E090E0F9
:100FD000A4E6B0E08D939C9306B30F3B09F011C0DB
:100FE000E2EDF5E1C8D4B3D206B30F3B09F4F8CF74
:100FF000E8E1F6E1C0D480E090E0A4E6B0E08D93B3
:101000009C9306B30F3709F011C0EAEDF5E1B3D4B4
:101010009ED206B30F3709F4F8CFE8E2F6E1ABD47D
:1010200080E090E0A4E6B0E08D939C938199A2C00B
:1010300006B30E3F09F00EC0E0E6F6E19CD487D27D
:1010400006B30E3F09F4F8CF80E090E0A4E6B0E0EC
:101050008D939C9306B30D3F09F00EC0E2E7F6E1D5
:101060008AD475D206B30D3F09F4F8CF80E090E042
:10107000A4E6B0E08D939C9306B30B3F09F00EC03D
:10108000E2EBF6E178D463D206B30B3F09F4F8CF74
:1010900080E090E0A4E6B0E08D939C9306B3073F18
:1010A00009F017C0EEEEF6E166D4ECE8F5E163D4A2
:1010B0004ED206B3073F09F4F8CFE8EAF5E15BD476
:1010C000E0EFF6E158D480E090E0A4E6B0E08D9344
:1010D0009C9306B30F3E09F017C0EEEEF6E14BD439
:1010E000E2E9F5E148D433D206B30F3E09F4F8CF74
:1010F000E4EBF5E140D4E0EFF6E13DD480E090E0B0
:10110000A4E6B0E08D939C9306B30F3D09F00EC0AA
:10111000E4ECF6E130D41BD206B30F3D09F4F8CF6E
:1011200080E090E0A4E6B0E08D939C9306B30F3B83
:1011300009F00EC0ECE7F6E11ED409D206B30F3B6E
:1011400009F4F8CF80E090E0A4E6B0E08D939C93A2
:1011500006B30F3709F00EC0EAE9F6E10CD4F7D177
:1011600006B30F3709F4F8CF80E090E0A4E6B0E0D2
:101170008D939C937FEE75BB8699A2C006B30E3FFC
:1011800009F017C0E4EFF6E1F6D3EAEEF5E1F3D3A8
:10119000DED106B30E3F09F4F8CFE8E4F6E1EBD375
:1011A000E6EFF6E1E8D380E090E0A4E6B0E08D93CE
:1011B0009C9306B30D3F09F017C0E4EFF6E1DBD3D3
:1011C000ECECF5E1D8D3C3D106B30D3F09F4F8CF69
:1011D000ECE0F6E1D0D3E6EFF6E1CDD380E090E0AD
:1011E000A4E6B0E08D939C9306B30B3F09F017C0C3
:1011F000E4EFF6E1C0D3E6EEF5E1BDD3A8D106B346
:101200000B3F09F4F8CFE0E4F6E1B5D3E6EFF6E101
:10121000B2D380E090E0A4E6B0E08D939C9306B357
:101220000F3D09F017C0E4EFF6E1A5D3E2EFF5E1D9
:10123000A2D38DD106B30F3D09F4F8CFE8E5F6E16E
:101240009AD3E6EFF6E197D380E090E0A4E6B0E031
:101250008D939C9306B30F3B09F017C0E4EFF6E1C2
:101260008AD3EEECF5E187D372D106B30F3B09F4D4
:10127000F8CFE0E1F6E17FD3E6EFF6E17CD380E062
:1012800090E0A4E6B0E08D939C9306B30F3709F08D
:1012900017C0E4EFF6E16FD3E2ECF5E16CD357D180
:1012A00006B30F3709F4F8CFE8EFF5E164D3E6EFC2
:1012B000F6E161D380E090E0A4E6B0E08D939C93EA
:1012C000A0E3B0E00C9101FB81E00EF080E08F9391
:1012D000A0E3B0E00C9105FB81E00EF080E09F916F
:1012E00089238F93A0E3B0E00C9106FB81E00EF020
:1012F00080E09F918923882309F4A8C006B30E3F9C
:1013000009F011C0EAEEF5E136D321D106B30E3F64
:1013100009F4F8CFE8E4F6E12ED380E090E0A4E60B
:10132000B0E08D939C9306B30D3F09F011C0ECEC37
:10133000F5E121D30CD106B30D3F09F4F8CFECE071
:10134000F6E119D380E090E0A4E6B0E08D939C93A1
:1013500006B30B3F09F011C0E6EEF5E10CD3F7D070
:1013600006B30B3F09F4F8CFE0E4F6E104D380E0E4
:1013700090E0A4E6B0E08D939C9306B3073F09F09C
:1013800011C0EEE8F5E1F7D2E2D006B3073F09F469
:10139000F8CFECEAF5E1EFD280E090E0A4E6B0E02F
:1013A0008D939C9306B30F3E09F011C0E0E9F5E17F
:1013B000E2D2CDD006B30F3E09F4F8CFE0EBF5E171
:1013C000DAD280E090E0A4E6B0E08D939C9306B37F
:1013D0000F3D09F011C0E2EFF5E1CDD2B8D006B370
:1013E0000F3D09F4F8CFE8E5F6E1C5D280E090E0E2
:1013F000A4E6B0E08D939C9306B30F3B09F011C0B7
:10140000EEECF5E1B8D2A3D006B30F3B09F4F8CF68
:10141000E0E1F6E1B0D280E090E0A4E6B0E08D93A8
:101420009C9306B30F3709F011C0E2ECF5E1A3D2AB
:101430008ED006B30F3709F4F8CFE8EFF5E19BD271
:1014400080E090E0A4E6B0E08D939C9381997EC00B
:1014500006B30E3F09F00EC0E8ECF6E18CD277D06F
:1014600006B30E3F09F4F8CF80E090E0A4E6B0E0C8
:101470008D939C9306B30B3F09F00EC0EAEBF6E1A7
:101480007AD265D006B30B3F09F4F8CF80E090E044
:10149000A4E6B0E08D939C9306B3073F09F017C014
:1014A000EEEEF6E168D2EEE8F5E165D250D006B393
:1014B000073F09F4F8CFECEAF5E15DD2E0EFF6E1A1
:1014C0005AD280E090E0A4E6B0E08D939C9306B3FE
:1014D0000F3E09F017C0EEEEF6E14DD2E0E9F5E17E
:1014E0004AD235D006B30F3E09F4F8CFE0EBF5E170
:1014F00042D2E0EFF6E13FD280E090E0A4E6B0E037
:101500008D939C9306B30F3D09F00EC0E4EEF6E117
:1015100032D21DD006B30F3D09F4F8CF80E090E041
:10152000A4E6B0E08D939C9306B30F3709F00EC08C
:10153000ECE5F6E120D20BD006B30F3709F4F8CF73
:1015400080E090E0A4E6B0E08D939C93ADC5A4E666
:10155000B0E00D911C91013050E0150709F006C074
:10156000A2E6B0E08D919C910AD10BC0A0E6B0E05C
:101570008D919C9104D181E090E0A4E6B0E08D9340
:101580009C93089501450116011E01260125012E97
:101590000136013D013E014602F0450002F0160011
:1015A00002F01E0002F0260002F0250002F02E00DC
:1015B00002F0360002F03D0002F03E0002F046006C
:1015C000011C0132012101230124012B01340133CB
:1015D0000143013B0142014B013A01310144014DFC
:1015E0000115012D011B012C013C012A011D0122C5
:1015F000011A013502F01C0002F0320002F0210055
:1016000002F0230002F0240002F02B0002F034006C
:1016100002F0330002F0430002F03B0002F042000F
:1016200002F04B0002F03A0002F0310002F04400F8
:1016300002F04D0002F0150002F02D0002F01B0038
:1016400002F02C0002F03C0002F02A0002F01D0023
:1016500002F0220002F01A0002F03500034AF04ABC
:101660000341F04105E069E0F06906595BF059F08B
:101670005B0005E06CE0F06C0361F0610812E07162
:10168000E0F071F012000812E070E0F070F012006B
:1016900008E01161E0F011F0610006594AF059F0DC
:1016A0004A00065961F059F0610006594EF059F0B0
:1016B0004E00035BF05B030DF00D08E0115BE0F002
:1016C00011F05B00035DF05D0349F04906595DF0E0
:1016D00059F05D00065949F059F04900065941F0AA
:1016E00059F0410008E0114EE0F011F04E000159B0
:1016F00002F05900011202F0120002F0140001146D
:10170000061421F014F02100061405F014F0050071
:10171000061406F014F00600061404F014F0040099
:1017200006140CF014F00C0002E0720002E07400E9
:1017300002E0750002E06B0003E0F07203E0F07479
:1017400003E0F07503E0F06B0329F029035AF05A27
:101750000376F0760366F0660305F0050306F006EF
:101760000304F004030CF00C0307F0073197F1F7C2
:101770000895689462F80895E89462F80895EF93E4
:10178000FF93EE27E82BE92B31F0E4EFF1E03197FE
:10179000F1F70197D1F7FF91EF9108958AEA00C020
:1017A000E8941FB6F894879BFECFEF93FF93E5E193
:1017B000F0E0DCDFFF91EF91879BF5CF839B20C0AA
:1017C000EF93FF93E6E0F0E0D1DFFF91EF9198E037
:1017D00088941AD0AEF00024879516D08EF09A9592
:1017E000D9F7889400FE08940FD056F008940CD0D6
:1017F0003EF0EF93FF93EBE0F0E0B8DFFF91EF9165
:10180000882780F91FBE089510F08B9A02C08B982C
:101810000394EF93FF93E6E0F0E0A8DFFF91EF91F0
:101820008F9AEF93FF93E0E1F0E0A0DFFF91EF915B
:101830008F98EF93FF93E6E0F0E098DFFF91EF9150
:101840008B98879B6894000008951FB6F89468945D
:1018500000248827879BFECF839967C098E0EF9389
:10186000FF93E6E0F0E082DFFF91EF918F9AEF9334
:10187000FF93E3E1F0E07ADFFF91EF918F98EF9330
:10188000FF93E6E0F0E072DFFF91EF918894839B95
:1018900002C00394089487959A9509F792E0EF9314
:1018A000FF93E6E0F0E062DFFF91EF918F9AEF9314
:1018B000FF93E0E1F0E05ADFFF91EF918F98EF9313
:1018C000FF93E6E0F0E052DFFF91EF918894839977
:1018D000089407959A9519F7EF93FF93E4E0F0E0E9
:1018E00045DFFF91EF918B9AEF93E5E0EA95F1F7F1
:1018F000EF918F9AEF93FF93E0E1F0E037DFFF91F4
:10190000EF918F98EF93E5E0EA95F1F7EF918B98DF
:10191000EF93FF93E3E1F0E029DFFF91EF9106FD04
:10192000039400FCE894992790F91FBE08958DDF79
:10193000992309F00895823F21F48BEA31DF83E88F
:101940002FCF8E3E09F42CCF8F3F19F48AEF28DF7A
:1019500025CF8AEF25CF0F921F920F938F939F93DE
:101960008FB78F93E4DF8F918FBF9F918F910F91EE
:101970001F900F9018951F930AD0102D08D0802D1E
:101980000FDF992311F41A95C9F71F910895C8958F
:06199000319600200895CD
:00000001FF
